:020000020000FC
:020000005EC0E0
:020018005BC1CA
:0200900074C139
:1000BC009CC001E20EBF0FEF0DBF07E104B908E0D1
:1000CC0005B901E00DBD00E50CBD289A2C980F9ADE
:1000DC0017980000179A0CE000936A0000E20DBB21
:1000EC0040E8E5D08FD003EC2898DBD001E0D9D0E4
:1000FC00289A000000000000000000000000000032
:10010C0000000000000000000000000000000000E3
:10011C005FEFCDD00BEE009364000EE10093650011
:10012C0000E900BF00EE2898BCD004E4BAD0289AAD
:10013C0001EE2898B6D004E4B4D0289A02EE2898A0
:10014C00B0D003ECAED0289A03EE2898AAD004EADB
:10015C00A8D0289A08EC2898A4D003E3A2D0289A17
:10016C0005EC28989ED000E89CD0289A0CEE289894
:10017C0098D00EE096D0289A0EEE289892D002E0F5
:10018C0090D0289A0DEE28988CD000E28AD0289A2C
:10019C000FE8289886D0289A0EEC289882D008E090
:1001AC0080D0289A08E90093C90001E00093CC00A4
:1001BC00B2E0AA27ED01002700932101009325014D
:1001CC000093240107E20093290100E10093280128
:1001DC0002E00ABB009373000FEF0CBB789443D082
:1001EC000000000000000000FBCF0F930FB70F932F
:1001FC000027009321010093730093D00F910FBF40
:10020C000F91189502EC28984CD008E04AD0289A07
:10021C0001E8289846D000E044D0289A0830C1F76D
:10022C00089502EC28983DD003E03BD0289A0000BA
:10023C0000000000000001E8289833D000E031D025
:10024C00289A083071F7089502EC28982AD009E012
:10025C0028D0289A01E8289824D000E022D0289AA7
:10026C000930C1F7089502EC28981BD009E119D088
:10027C00289A01E8289815D000E013D0289A093163
:10028C00C1F7089502EC28980CD006E10AD0289A00
:10029C0001E8289806D000E004D0289A0631C1F76E
:1002AC0008950EBD0DB507FFFDCF0EB508950000E6
:1002BC0000000000000000000000000000004A9553
:1002CC00B1F708950F930FB70F930FE82898E9DF54
:1002DC00289A01E82898E5DF00E0E3DF289A0F313F
:1002EC00C1F30231B1F30931B1F402E82898D9DF36
:1002FC0000E0D7DF289A007E003348F0C22FFA9432
:10030C0010D000270093210102E00ABB06C002E0D6
:10031C000093730002C085DFA6DF0F910FBF0F9112
:10032C0018952C9A00002C9800E62898BADF2C2FF0
:10033C003A2F321B0BE0030FB4DF01E6B2DF08E803
:10034C00B0DFF3940F2DADDF03ECABDF04EAA9DFD4
:10035C0006E6A7DF06E6A5DF04E4A3DF04E4A1DFDD
:10036C000991D2709EDF3A95D9F7289A08950F9388
:10037C000FB70F930091CE000D93B2700091210135
:10038C000770013058F400270093250100932401D5
:10039C0001E00093210102E0009373000F910FBF65
:0403AC000F91189500
:00000001FF
